:100000003828FF3FFF3FFF3F03138312A201A301E4
:100010008613A401A501A60108000B1D0D280B11D4
:100020006130031383128102A50A0319A60A08008E
:1000300000300313831698180130F1007108003A5C
:10004000031D24280000182883123A08990008008C
:100050000313831698169030831298008316861423
:10006000061183128C1E37281A08BE00312808009A
:100070001E30031383129F00E53083169F00831206
:10008000850115308316850083128601083083169A
:10009000860088308100013083129000053097007F
:1000A000042081308316990018152820A501A60187
:1000B000A701C830270203186C280D208619612873
:1000C000A70101302602031D6728F4302502031C16
:1000D0006A280420A70A5928A501A601A7010A3009
:1000E0002702031882280D20861D7728A7010130DA
:1000F0002602031D7D28F4302502031C80280420DD
:10010000A70A6F28A501A6010C110C1992280D2031
:1001100000302602031D8E2864302502031C91281E
:10012000042085281508A0001608A1002A0820022E
:10013000F1002B08031C013F2102F2007108A80006
:100140007208A9002008AA002108AB009C307202A6
:10015000031DAC283F307102031CB6282908A93CB6
:10016000031DB4282808443C0318B8280420BF28DD
:10017000A20A2208C83C0318BF28C830A200643075
:100180002202031C3B29B10D31100030B01B01309D
:10019000F10000307118013031060139B106B00D9F
:1001A00030100030AF1B0130F10000307118013009
:1001B00030060139B006AF0D2F100030AE1B0130F4
:1001C000F1000030711801302F060139AF06AE0D75
:1001D0002E100030AD1B0130F100003071180130DD
:1001E0002E060139AE06AD0D2D100030AC1B0130CE
:1001F000F1000030711801302D060139AD06AC0D4B
:100200002C100030A0180130F100003071180130BE
:100210002C060139AC06B50D35100030B41B013089
:10022000F10000307118013035060139B506B40D02
:1002300034100030B31B0130F10000307118013070
:1002400034060139B406B30D33100030B21B01304F
:10025000F10000307118013033060139B306B20DD8
:100260003210003020190130F100003071180130D7
:1002700032060139B2062208933C03187129013075
:100280002005F00000307018013038060139B8063A
:10029000B11F4C290130B806B51E50290130B806EF
:1002A000B90D391001303805F000003070180130F8
:1002B00039060139B906A30A08302302031C642950
:1002C000A3013908BA001820A40A78302402031CBC
:1002D0006A29A4013C302402031870298617712969
:1002E000861356287229FF3FFF3FFF3FFF3FFF3F26
:02400E00023F6F
:00000001FF
